:100000000C9403050C9420050C9420050C942005F9
:100010000C9420050C9420050C9420050C942005CC
:100020000C9420050C9420050C9416260C94E826BC
:100030000C945F200C9420050C9420050C94200552
:100040000C9420050C9420050C9420050C9420059C
:100050000C9420050C94E7200C9420050C942005AA
:100060000C9420050C9420050C9420050C9420057C
:100070000C9420050C9420050C9420050C9420056C
:100080000C9420050C9420050C9420050C9420055C
:100090000C9420050C9420050C9420050C9420054C
:1000A0000C9420050C9420050C942005DB08DB083B
:1000B000070907096F098D09A50AA50A9809310AD8
:1000C000420A420A55277C2774287C277428C827AF
:1000D000EB27742842285128105011501250240048
:1000E000250026002100220023001E001F00200002
:1000F00027002A0028001050115012504A005200C8
:100100004B00500029004F004D0051004E004C00A4
:100110002A0028001050115012507B007C007D00F6
:100120007A007E0079000000000000004C002A00E8
:10013000280044454255473A2064697361626C6502
:10014000642E0A0044454255473A20656E61626C50
:1001500065642E0A000A0025303258006C65645F21
:100160007461736B3A20004F6E6573686F743A2048
:100170006163746976653A2025640A000A002530B7
:100180003862003A200025303258000A722F63206E
:1001900030313233343536370A00290A00257500EC
:1001A0002F002575005D28002564002000256400CF
:1001B000200025640020002564007C002530325892
:1001C000006D6F7573656B6579205B62746E7C780A
:1001D0002079207620685D287265702F61636C2914
:1001E0003A205B00313A0964656C6179282A313024
:1001F0006D73293A2025750A323A09696E74657261
:1002000076616C286D73293A2025750A333A096D99
:1002100061785F73706565643A2025750A343A0920
:1002200074696D655F746F5F6D61783A2025750A3A
:10023000353A09776865656C5F6D61785F737065E5
:1002400065643A2025750A363A09776865656C5FFA
:1002500074696D655F746F5F6D61783A2025750A0A
:1002600000703A097072696E742076616C756573FE
:100270000A643A097365742064656661756C747309
:100280000A75703A092B310A646E3A092D310A6CED
:10029000743A092B31300A72743A092D31300A450B
:1002A00053432F713A09717569740A0A7370656551
:1002B00064203D2064656C7461202A206D61785F44
:1002C0007370656564202A202872657065617420EA
:1002D0002F2074696D655F746F5F6D6178290A778F
:1002E000686572652064656C74613A206375727329
:1002F0006F723D25642C20776865656C3D25640A26
:1003000053656520687474703A2F2F656E2E776977
:100310006B6970656469612E6F72672F77696B69AD
:100320002F4D6F7573655F6B6579730A004D3E20C5
:10033000004D25753A25733E20003F0A003D2025DB
:10034000750A003F0A0064656661756C74730A0083
:1003500025750A003F0A000A092D2056616C756553
:1003600073202D0A00710A000A092D204D6F757344
:10037000656B6579202D0A003F00433E20004C2527
:10038000640A000A092D20537461747573202D0AC4
:10039000686F73745F6B6579626F6172645F6C65BF
:1003A000647328293A20253032580A6B6579626FC8
:1003B0006172645F70726F746F636F6C3A20253086
:1003C00032580A6B6579626F6172645F69646C654B
:1003D0003A20253032580A74696D65725F72656122
:1003E00064333228293A202530386C580A000A092B
:1003F0002D2056657273696F6E202D0A5649443A56
:100400002030784645454428542E5368696E6F68FD
:1004100061726129205049443A20307830303030C0
:1004200028536869726F29205645523A2030783037
:100430003030310A4255494C443A20202846656202
:100440002032382032303232290A4F5054494F4E30
:10045000533A204C554641204D4F5553454B455935
:100460002045585452414B455920434F4E534F4C11
:100470004520434F4D4D414E4420343039360A47D4
:1004800043433A20352E342E30204156522D4C49CC
:1004900042433A20322E302E30204156525F415294
:1004A00043483A20617672350A000A092D20436FCD
:1004B0006E736F6C65202D0A4553432F713A097195
:1004C0007569740A6D3A096D6F7573656B65790AA4
:1004D000000A092D204D61676963202D0A443A09FD
:1004E0004465627567204D65737361676520546F5D
:1004F00067676C650A583A094D61747269782044DF
:1005000065627567204D6F646520546F67676C6521
:10051000202D2053686F77206B6579707265737337
:10052000657320696E206D617472697820677269E5
:10053000640A4B3A094B6579626F617264204465C5
:1005400062756720546F67676C65202D2053686F54
:1005500077206B65797072657373207265706F7246
:10056000740A4D3A094465627567204D6F7573656D
:1005700020546F67676C650A563A0956657273694D
:100580006F6E0A533A095374617475730A433A09DA
:10059000416374697661746520436F6E736F6C6537
:1005A000204D6F64650A46312D4631303A09537744
:1005B0006974636820746F204C6179657220302DF6
:1005C000392028463130203D204C30290A302D3941
:1005D0003A0953776974636820746F204C617965B8
:1005E0007220302D390A47524156453A09537769EE
:1005F00074636820746F204C617965722030202804
:10060000616C7465726E617465290A423A094A75B3
:100610006D7020746F20426F6F746C6F61646572CF
:100620000A4553433A094A756D7020746F20426F32
:100630006F746C6F616465722028616C7465726E92
:10064000617465290A453A095072696E74204545FE
:1006500050524F4D2053657474696E67730A42534C
:10066000504143453A09436C6561722045455052FB
:100670004F4D0A006B65796D61705F636F6E6669DF
:10068000672E7261773A20253032580A2E737761CF
:10069000705F636F6E74726F6C5F636170736C6FA9
:1006A000636B3A2025750A2E636170736C6F636B00
:1006B0005F746F5F636F6E74726F6C3A2025750A9A
:1006C0002E737761705F6C63746C5F6C6775693AE9
:1006D0002025750A2E737761705F7263746C5F7288
:1006E0006775693A2025750A2E737761705F6C61B2
:1006F0006C745F6C6775693A2025750A2E73776193
:10070000705F72616C745F726775693A2025750A53
:100710002E6E6F5F6775693A2025750A2E737761B3
:10072000705F67726176655F6573633A2025750A4D
:100730002E737761705F6261636B736C6173685F66
:100740006261636B73706163653A2025750A2E6E72
:100750006B726F3A2025750A0064656275675F6386
:100760006F6E6669672E7261773A20253032580ABB
:100770002E656E61626C653A2025750A2E6D617476
:100780007269783A2025750A2E6B6579626F6172FD
:10079000643A2025750A2E6D6F7573653A202575AC
:1007A0000A006565636F6E6669673A0A646566612B
:1007B000756C745F6C617965723A2025750A003F2B
:1007C000000A6D6F7573653A206F66660A000A6DE0
:1007D0006F7573653A206F6E0A000A6B6579626FF8
:1007E0006172643A206F66660A000A6B6579626F0F
:1007F0006172643A206F6E0A000A6D6174726978E2
:100800003A206F66660A000A6D61747269783A2050
:100810006F6E0A000A64656275673A206F66660A41
:10082000000A64656275673A206F6E0A000A0A4A18
:10083000756D70696E6720746F20626F6F746C6F76
:10084000616465722E2E2E2000433E2000436C65AD
:100850006172696E6720454550524F4D0A000A008B
:100860002530325820006B6579626F6172645F7267
:1008700065706F72743A20005B735D005B575D00BA
:100880005B535D005B525D005B445D005B435D005C
:100890000C0353006800690072006F000000180329
:1008A00054002E005300680069006E006F0068005D
:1008B00061007200610000000403090409025B008A
:1008C000030100A0FA09040000010301010009214D
:1008D00011010001224000070581030800010904FD
:1008E00001000103000000092111010001227B0029
:1008F0000705820320000109040200020300000032
:1009000009211101000122220007058303200001B3
:10091000070503032000011201000200000008ED9A
:10092000FE00000100010200010631FF0974A1016F
:100930000975150026FF00952075088102097615B6
:100940000026FF00952075089102C005010902A14B
:100950000185020901A100050919012908150025D1
:1009600001950875018102050109300931158125BC
:100970007F95027508810609381581257F950175D7
:10098000088106050C0A38021581257F9501750836
:100990008106C0C005010980A101850319012AB79C
:1009A00000150126B700950175108100C0050C09DE
:1009B00001A101850419012AA002150126A00295B2
:1009C0000175108100C005010906A101050719E0A4
:1009D00029E7150025019508750181029501750823
:1009E00081010507190029FF150026FF00950675EE
:1009F00008810005081901290595057501910295E1
:100A00000175039101C011241FBECFEFDAE0DEBFF4
:100A1000CDBF11E0A0E0B1E0E4E6F2E502C0059050
:100A20000D92A03FB107D9F722E0A0EFB1E001C0DD
:100A30001D92AF3AB207E1F70E94B7160C94302925
:100A40000C940000FF93EF93E091F001F091F1011D
:100A5000309709F00995EF91FF910895FC01859178
:100A6000803011F0EFDFFBCF0895FF27E0E230E2A6
:100A700047FF0CC0419597FF09C0EDE26095709566
:100A800080959095611D711D811D911D27FF02C0EC
:100A9000219530E350E2AA27660F771F881F991F20
:100AA000AA1FA41710F0A41B63955A95A9F7AA30A2
:100AB00008F0A95FA05DAF93F395611571058105FD
:100AC000910541F7ED3211F4EF93F395F21718F415
:100AD0003F93F395FBCF8F91B5DFFA95E1F708953A
:100AE000E991F9918591803021F0853219F0AADFE2
:100AF000F9CF089520E0E89455915532C1F3503371
:100B000011F4689455915A3348F4505390F3220FDE
:100B1000022E220F220F200D250FF4CF0EF4219567
:100B200089919991533619F3533729F1533559F176
:100B3000BC0188279927E8945C3621F48991999122
:100B400068945591543639F446EF7EF077FF0DC026
:100B50008FEF9FEF0AC055374AE039F0583540E132
:100B600021F0523642E009F00895FF93EF937DDFC4
:100B7000EF91FF91B7CFFF93EF93FC01819180300C
:100B8000B9F360DFFBCFFF93EF9368DFF1CFDF9323
:100B9000CF93CDB7DEB72596A3DFCF91DF91089530
:100BA00081E0089581E008950C94D20508950C9495
:100BB000D6051F93CF93DF9300D000D01F92CDB7FF
:100BC000DEB749835A836B833091F30189819A811F
:100BD000311114C0662359F0222349F00E94E20C1F
:100BE000182F682F89819A810E948B0C03C00E9464
:100BF000B60C182F69817A81812F04C00E94E20C03
:100C000069817A810F900F900F900F900F90DF9174
:100C1000CF911F910C941114FC01262F408151811A
:100C20006281738184810C94D90581E00895CF930A
:100C3000DF93EC0160E00E940C06BE01DF91CF91D2
:100C40000C94D7050C9483150C947F1508950E947D
:100C5000350B0E9426062FEF84E39CE02150804054
:100C60009040E1F700C000000C940D210F931F93FA
:100C7000CF93DF938C0161E00E940C06EC01B80178
:100C80000E94D405882309F45BC0B801CE010E94FC
:100C9000ED1E882309F454C0B801CE010E94CF197B
:100CA000882309F44DC0B801CE010E94491E882353
:100CB00009F446C0F80182818823D9F1CF3D8CE543
:100CC000D80779F140F4C115FCE5DF0791F0C13098
:100CD000DC4591F02EC0CC35EDE5DE0741F1CD3598
:100CE000FDE5DF0709F1CB35DD4519F50E947911E6
:100CF00020C00E94270624C080915F02C82FC095A3
:100D0000C170C0FB80F980935F02CC2329F084E49A
:100D100091E00E942E0514C082E391E00E942E050E
:100D200010C00E9427120CC00E94701102C00E94C5
:100D30007C11C801DF91CF911F910F910C94D005C8
:100D4000C0E08C2FDF91CF911F910F9108950E94E9
:100D500042200C94D2060E94D5060C94482082951D
:100D6000982F937344E0949F900111248C7C869576
:100D70008695282B822F8575880F2A7A2695822BB7
:100D8000089508950C94C10681E008950C94C4065A
:100D90000895CF93C82F0E94C2068C2F0E94C606CA
:100DA000CF91089580E00C94C9060E94491F0C94CD
:100DB000C906CF930E94491FC82F8091F201C8171E
:100DC00041F1C093F20180915F0282FF1EC080FF5B
:100DD00004C08CE591E00E942E0580915F0280FFA7
:100DE0000CC01F92CF9387E591E09F938F930E9451
:100DF000C7050F900F900F900F9080915F0280FFBA
:100E000004C085E591E00E942E058C2FCF910C94B3
:100E1000C906CF910895CF93DF93CDB7DEB72B9757
:100E20000FB6F894DEBF0FBECDBF4F8358876987DA
:100E30007A878B8761110E94A8109E012F5F3F4F18
:100E400086E0F90111928A95E9F785E0FE0137966F
:100E5000D90101900D928A95E1F789819A814C819F
:100E60005D81452B31F09F3F31F491E08F3F19F4C4
:100E700003C091E001C090E090FF09C049815A8110
:100E80006B817C818D819E810E94C90F05C0C90143
:100E90000E9415068111F2CF2B960FB6F894DEBF93
:100EA0000FBECDBFDF91CF910895FC01808191816C
:100EB0000E94240D0895CF93882309F4A9C0C82F58
:100EC0008238C1F40E94491F81FDA2C069E380916C
:100ED0000201909103010E941A200E94CA102FEF74
:100EE00081EE94E0215080409040E1F700C0000086
:100EF00069E319C0833801F50E94491F80FD88C04D
:100F000063E580910201909103010E941A200E94E2
:100F1000CA102FEF81EE94E0215080409040E1F71D
:100F200000C0000063E580910201909103010E94DE
:100F30001C20CF910C94CA108438C1F40E94491F20
:100F400082FD66C067E480910201909103010E94D6
:100F50001A200E94CA102FEF81EE94E021508040A9
:100F60009040E1F700C0000067E4DDCF8CEF8C0F0C
:100F7000813AF8F48C2F0E94F21D811149C06C2F28
:100F800080910201909103010E94E41F882349F09F
:100F90006C2F80910201909103010E941C200E94FD
:100FA000CA106C2F80910201909103010E941A20B7
:100FB000C0CF80E28C0F883048F4C77081E001C058
:100FC000880FCA95EAF70E948B10B3CFEBE5EC0FC0
:100FD000E33040F4F0E0E95BFE4F808190E0CF9198
:100FE0000C94AC1FE8E5EC0FE73150F4F0E0EE0FA5
:100FF000FF1FE75EFE4F80819181CF910C94C21F4D
:10100000CD3E30F08C2F0E943C17CF910C940E18DF
:10101000CF910895882309F464C0823879F40E943E
:10102000491F81FF5EC069E3809102019091030135
:101030000E941A200E94CA1069E310C08338B1F4DC
:101040000E94491F80FF4DC063E58091020190918D
:1010500003010E941A200E94CA1063E580910201D8
:10106000909103010E941C200C94CA10843879F4DA
:101070000E94491F82FF35C067E480910201909170
:1010800003010E941A200E94CA1067E4E7CF9CEF78
:10109000980F913A10F4682FE1CF90E2980F9830B2
:1010A00050F4877091E001C0990F8A95EAF7892F73
:1010B0000E949110D9CF9BE5980F933020F480E0E7
:1010C00090E00C94AC1F98E5980F973120F480E0E5
:1010D00090E00C94C21F8D3E20F00E9497170C9454
:1010E0000E1808951F93CF93DF93182FEB010E94E2
:1010F0005B07209741F08FE99FE00197F1F700C06F
:1011000000002197F6CF812FDF91CF911F910C9492
:101110000A08893319F060E070E002C060E570E011
:101120000C947208882321F00E948B100C94CA1032
:101130000895882321F00E9491100C94CA100895FC
:10114000CF92DF92EF92FF920F931F93CF93DF9393
:101150007C01D62FC72FFC011281058102950F70EB
:101160000E9481108823B9F01123A9F08C2F807F71
:10117000803421F080E28D0F883068F080919302F6
:1011800082FD09C082E00E942A110E94811091E034
:10119000D82ED92601C0D12CCC2EC2948FE0C822E3
:1011A0008C2D90E08C30910508F0CFC1FC01EA5AFB
:1011B000FF4F0C94C7288C2F807FCF70882311F0AD
:1011C000C295C07F112399F0CC2309F4AAC180E213
:1011D0008D0F883010F0D11104C08C2F0E948B101D
:1011E00003C08C2F0E949B100E94CA109AC18D2FA1
:1011F0000E940A08CC2309F4A8C180E28D0F883030
:1012000038F1DD2329F18C2F0E94A11024C08C2FEE
:10121000807FCF70803211F0C295C07FDD2319F03E
:10122000D130A1F13DC08091930282FF17C01123FC
:1012300049F0CC2329F08C2F0E948B100E94CA10F9
:1012400080E070C180E00E940A08CC2309F47DC1CF
:101250008C2F0E9491100E94CA1077C1112371F047
:10126000002341F0013031F40E94AB108C2B0E941E
:10127000B3106BC10E94AB108C2B1DC0002319F062
:10128000013009F462C10E94C01025C0112321F071
:10129000063008F05AC10EC0053008F056C11BC018
:1012A000112361F0002331F0F701858180FF39C1FE
:1012B0008F7085838C2F0E94920847C1002359F0BC
:1012C000D93309F03FC1FFEF07EE13E0F1500040C2
:1012D0001040E1F735C18C2F0E94990836C18C2F40
:1012E00086958695837019F0813061F02EC11123A7
:1012F00021F08D2F9C2F937002C080E090E00E941F
:10130000AC1F2BC1112321F08D2F9C2F937002C095
:1013100080E090E00E94C21F20C18D2F112319F0A0
:101320000E943C1702C00E9497170E940E1815C118
:101330008C2F837009F047C011110BC12D2F2295FE
:1013400026952770220F220F6D2F6F70862F90E049
:10135000A0E0B0E0022E04C0880F991FAA1FBB1F97
:101360000A94D2F7D4FF10C04FE050E060E070E084
:1013700004C0440F551F661F771F2A95D2F740956A
:1013800050956095709503C040E050E0BA01C69555
:10139000C695C3708A019B01082B192B2A2B3B2B66
:1013A000C901B801C23049F058F4C13019F00E94A7
:1013B000A10BCFC00E948F0BCCC00E94B30BC9C041
:1013C0000E948D0BC6C0112319F08C2F817001C0B3
:1013D0008695882309F4BDC02D2F22952695277068
:1013E000220F220F6D2F6F70862F90E0A0E0B0E0EB
:1013F000022E04C0880F991FAA1FBB1F0A94D2F7A0
:10140000D4FF10C04FE050E060E070E004C0440F33
:10141000551F661F771F2A95D2F740955095609506
:10142000709503C040E050E0BA01C695C695C37000
:101430008A019B01082B192B2A2B3B2BC901B801D0
:10144000C23049F058F4C13019F00E94660C81C0D6
:101450000E94540C7EC00E94780C7BC00E94C70B77
:1014600078C0CF70112339F08C2F0E94ED0B8D2F97
:101470000E9492086EC08D2F0E9499088C2F0E94A6
:101480000E0C67C0D23F21F128F4D03F41F0D13F8C
:10149000C1F043C0D33F19F1D43F79F03EC01123CE
:1014A00041F0053008F051C08C2F8F710E94330C31
:1014B0004CC0063008F049C0F7CF8091930282FFFC
:1014C00018C0112339F08C2F8F710E94ED0B3DC095
:1014D0001123C9F38C2F8F710E940E0C36C011237B
:1014E00029F08C2F8F710E94D80B2FC00E94D30B34
:1014F0002CC0112349F0CF718C2F0E94ED0B63E0BB
:101500008C2F0E940F1121C081E00E942A1102300D
:10151000E0F082E00E942A1118C0112331F000236C
:1015200091F28D2F0E945B0710C0002399F2D933EE
:1015300049F41FEF27EE33E0115020403040E1F72F
:1015400000C000008D2F0E940A0888EF8C0D8430A7
:1015500020F40E94491F0E94C906DD20C9F00E94A4
:101560007D1080FD15C0F70112820E9477100E9445
:10157000ED0BC7010E94E90A0E947710DF91CF911D
:101580001F910F91FF90EF90DF90CF900C940E0C75
:10159000DF91CF911F910F91FF90EF90DF90CF904F
:1015A00008950F931F93CF93DF93EC0168817981A6
:1015B0008A810E942F0D8C010E948A0C0E947B0B55
:1015C000B801CE010E94A008DF91CF911F910F9129
:1015D0000895CF93DF93EC01988189812B813C8121
:1015E000232B31F08F3F31F481E09F3F19F403C08A
:1015F00081E001C080E080FD1DC0CE010E94360662
:10160000811110C00E9481108823A1F08A81882353
:1016100089F08091930282FD0DC082E0DF91CF912D
:101620000C942A11CE010E94D10ACE01DF91CF91F4
:101630000C941706DF91CF91089580E090E00E940E
:10164000AC1F80E090E00E94C21F0E94A8100E9480
:10165000CA100E94C1190C940E1880910201909139
:1016600003010E941E200C941D0B0E9498100C94E4
:101670002D0B92959F70963079F010F4925001C026
:101680009A50923068F4803F69F018F4883E40F434
:1016900009C0843F29F406C0883E20F0813F11F044
:1016A00080E0089581E00895FC01808191810E948D
:1016B000240D0E94390B0895CF93DF9300D000D002
:1016C0001F92CDB7DEB70F900F900F900F900F9035
:1016D000DF91CF910895CF93DF9300D000D000D059
:1016E000CDB7DEB726960FB6F894DEBF0FBECDBFDE
:1016F000DF91CF910895089508950C947C0B0C947C
:101700007D0B0E947F0B6093020270930302809313
:101710000402909305020C941D0B0C94810B0F9303
:101720001F93009102021091030220910402309154
:101730000502602B712B822B932B1F910F910C9420
:10174000810B0F931F9300910202109103022091CD
:1017500004023091050260237123822393231F9199
:101760000F910C94810B0F931F9300910202109123
:10177000030220910402309105026027712782271D
:1017800093271F910F910C94810B0C947C0B0E945A
:10179000C50B6093FE017093FF018093000290934C
:1017A00001020C941D0B60E070E0CB010C94C70BA0
:1017B0000F931F9341E050E060E070E08A019B01CD
:1017C00004C0000F111F221F331F8A95D2F7C901D1
:1017D000B8011F910F910C94C70B0F931F9341E019
:1017E00050E060E070E004C0440F551F661F771F93
:1017F0008A95D2F78091FE019091FF01A09100029D
:10180000B09101028A019B01082B192B2A2B3B2B3B
:10181000C901B8011F910F910C94C70B0F931F932F
:1018200041E050E060E070E004C0440F551F661FC7
:10183000771F8A95D2F74095509560957095809165
:10184000FE019091FF01A0910002B09101028A0176
:101850009B01082319232A233B23C901B8011F91A7
:101860000F910C94C70B0F931F9341E050E060E081
:1018700070E004C0440F551F661F771F8A95D2F78A
:101880008091FE019091FF01A0910002B0910102B0
:101890008A019B01082719272A273B27C901B8017C
:1018A0001F910F910C94C70B0F931F930091FE0192
:1018B0001091FF012091000230910102602B712BE9
:1018C000822B932B1F910F910C94C70B0F931F9397
:1018D0000091FE011091FF01209100023091010260
:1018E00060237123822393231F910F910C94C70BC4
:1018F0000F931F930091FE011091FF0120910002B0
:101900003091010260277127822793271F910F9141
:101910000C94C70B0895292F220F920F890FE82FDF
:10192000E695E695E695877051E001C0550F8A95DA
:10193000EAF785E0E89FF0011124EC50FE4F20E02B
:1019400030E070E04081CB01022E02C09695879571
:101950000A94E2F7817081958427852384278193F7
:101960002F5F3F4F2530310569F70895292F220F4A
:10197000920F890F682F669566956695982F9770D8
:1019800085E0689FB001112440E050E080E0FB0159
:10199000E40FF51FEC50FE4F208130E0092E02C00D
:1019A000369527950A94E2F721703327042E01C05B
:1019B000220F0A94EAF7822B4F5F5F4F45305105A3
:1019C00031F70895BF92CF92DF92EF92FF920F937B
:1019D0001F93CF93DF938C01C090FE01D090FF0145
:1019E000E0900002F09001028091020290910302C7
:1019F000A0910402B0910502C82AD92AEA2AFB2A3A
:101A0000CFE1D0E0D701C6010C2E04C0B695A79552
:101A1000979587950A94D2F780FD04C0219790F797
:101A2000B12C07C0BC2EB8018C2F0E94271401973F
:101A3000A9F38B2DDF91CF911F910F91FF90EF9024
:101A4000DF90CF90BF900895CF93DF93EC010E9479
:101A5000E20CBE010E942714DF91CF9108951F93DD
:101A6000CF93DF93EB019091F301992321F0CB0108
:101A70000E94240D13C0882349F0CB010E94E20C80
:101A8000182F682FCE010E948B0C04C0CB010E943E
:101A9000B60C182FBE01812F0E942714DF91CF9121
:101AA0001F9108951F93CF93DF93C091060216E014
:101AB00080910702C81799F0D0E01C9FF0011D9F8C
:101AC000F00D1124E85FFD4F4081518162817381E7
:101AD000848195810E946B0B2196C770E9CFDF91BD
:101AE000CF911F9108954091380250913902609131
:101AF0003A0270913B0280913C0290913D020C941D
:101B00006B0BEF92FF920F931F93CF93DF93809114
:101B10003D0282958F7009F065C080913A0288235A
:101B200009F460C080910602F0900702109138021B
:101B30000091390260913B0270913C0291E01F3F9D
:101B400009F090E0C0910001D0910101292F96E0A9
:101B5000E92E8F1509F446C06115710521F00F3F7C
:101B600021F030E003C031E001C0322F90E030FDC1
:101B700036C0E89EF001E99EF00D1124DF01A85F58
:101B8000BD4F11963C911197301329C03C913113F0
:101B900026C012963C911297311121C013964D9197
:101BA0005C911497461B570B4C175D07C0F480914E
:101BB0003D028F70806180933D02E35FFD4F808125
:101BC0008F708061808388E392E00E94E90ADF9150
:101BD000CF911F910F91FF90EF900C94520D0196B1
:101BE0008770B7CFDF91CF911F910F91FF90EF904A
:101BF00008959F92AF92BF92CF92DF92EF92FF92A1
:101C00000F931F93CF93DF93CDB7DEB761970FB6D6
:101C1000F894DEBF0FBECDBF8C0185E0F801DE0178
:101C20001D9601900D928A95E1F7D8011296EC90DD
:101C300090913802E091390220913B0230913C02B0
:101C40002115310531F0EF3F31F481E09F3F19F468
:101C500003C081E001C080E0B82FB1709B2E80FDF1
:101C600047C1D8014C9111965C9111971396AD9094
:101C7000BC90149788E3C82E82E0D82EF0903A02E8
:101C8000B501621B730B2091000130910101FF200F
:101C900009F4D9C080913D026217730708F095C01E
:101CA000282F207F09F052C05E1313C0491311C0C2
:101CB000FE2CE1100EC08F70806180933D020E9467
:101CC000730DC6010E94E90A80913D02F8018583E7
:101CD0004DC1AB2831F05F3F31F481E04F3F19F443
:101CE00003C081E001C080E080FD03C081E08E255B
:101CF00002C080E090E0F82FF170FF2E80FF1CC042
:101D0000809106022091070236E0821709F40BC188
:101D100090E0389FF001399FF00D1124E85FFD4FEE
:101D20006181561306C06081461303C06281E612CA
:101D300003C001968770E9CFFE2CEE2009F416C18E
:101D400080913D02816080933D0254C05E1306C0C5
:101D5000491304C0E11002C0F80199C0C8010E94F3
:101D6000540B882361F1EE2051F120913D02822F26
:101D700082958F7090E0029774F080913802909174
:101D8000390298878F831986BB86AA862C87CE0155
:101D900007960E94E90A86E0F801A8E3B2E0019004
:101DA0000D928A95E1F70E94810D0E94730D0AC081
:101DB0005E1711F1C8010E94540B81112CC0C8019B
:101DC0000E94E90AFF24F394D1C0282F207F81F7D5
:101DD0007A2DB98AA88A6E2D89890E945C0B88E3C6
:101DE00092E00E94E90A86E0D6011D928A95E9F701
:101DF0000E94730DF12CBAC04913DCCFE110DACF89
:101E0000F8018583C8010E94E90A86E0D6011D9287
:101E10008A95E9F7ABC0EE2091F220913D02822F26
:101E200082958F7090E002970CF4B5CF80913802C4
:101E3000909139029A8389831B82BD82AC822E8362
:101E4000CE010196A6CF6217730708F044C0FE2C9E
:101E5000EE2009F4B4CF5E1330C049132EC0209198
:101E60003D0220FD21C0822F82958F70482F50E0C7
:101E700041155105C9F0F80125834F30510541F056
:101E80008F5F982F9295907F822F8F70892B8583FB
:101E9000C8010E94E90A86E0F801A8E3B2E00190D7
:101EA0000D928A95E1F73CC086E0F801A8E3B2E024
:101EB00001900D928A95E1F759C0C8010E94540B18
:101EC000811169CF80913D02816080933D02C801FC
:101ED0000E94E90A4BC07A2DB98AA88A6E2D898999
:101EE0000E945C0B86E0D6011D928A95E9F718C026
:101EF000EE2009F464CFC8010E94540BF82E882309
:101F000009F45DCF86E0F801A8E3B2E001900D92FC
:101F10008A95E1F788E392E00E9455070E94810DBF
:101F20000E94730D23C04D875E878D859E850E941C
:101F3000240D292F22952F70223028F49F7039F01C
:101F4000811105C00BC0243028F49F7049F4805ED5
:101F5000883020F0C8010E94E90A9F2CF92C06C0A5
:101F6000D80115969C91907F91F7F8CF8F2D6196AF
:101F70000FB6F894DEBF0FBECDBFDF91CF911F919A
:101F80000F91FF90EF90DF90CF90BF90AF909F9018
:101F900008951F93CF93DF93CDB7DEB72C970FB67D
:101FA000F894DEBF0FBECDBF4F83588769877A870D
:101FB0008B879C87CE0107960E94F90D8823D1F06C
:101FC0009F8188852A853B85232B31F08F3F31F413
:101FD00081E09F3F19F403C081E001C080E080FDF3
:101FE00047C04F81588569857A858B859C850E947D
:101FF0006B0B3EC086E0FE013796DE011196019024
:102000000D928A95E1F7FF81E8856A857B856115E8
:10201000710531F0EF3F31F481E0FF3F19F403C067
:1020200081E001C080E080FD23C02091070230E004
:10203000C9010196877099274091060250E08417E4
:102040009507F1F1F983EA837D836C8396E0929F93
:10205000D001939FB00D1124A85FBD4FFE013196B2
:1020600001900D929A95E1F7809307020E94520D1C
:1020700016E08091060290910702891771F1189F6E
:10208000C0011124885F9D4F0E94F90D882329F11A
:10209000E09106021E9FF0011124E85FFD4F408190
:1020A000518162817381848195810E946B0B809143
:1020B000060290E001968770992780930602D9CF97
:1020C0000E94350B1092070210920602E8E3F2E03C
:1020D00086E0DF011D928A95E9F72C960FB6F894F9
:1020E000DEBF0FBECDBFDF91CF911F9108958091CC
:1020F000460285958595859508958091460287705D
:10210000089590914602977081E009F480E0089567
:1021100080915102089590915102892B8093510230
:1021200008958095909151028923809351020895DA
:1021300010925102089590915002892B8093500281
:1021400008958095909150028923809350020895BC
:1021500010925002089580914702089508950C94BA
:10216000AE100C94AF109091930292FD08C0909124
:102170004702981721F0809347020C94B1100895FC
:1021800080914702882329F01092470280E00C9446
:10219000B1100895CF93DF93E0910201F091030114
:1021A000809151028083E0910201F09103019081BE
:1021B00080915002892B808380914702882381F08F
:1021C000E0910201F09103019081892B808380913D
:1021D0000201909103010E94D81F81110E94C0103A
:1021E000C0910201D091030148E050E06EE372E03B
:1021F000CE010E94E128892B69F088E0FE01AEE360
:10220000B2E001900D928A95E1F7CE01DF91CF9176
:102210000C94551FDF91CF9108950C94AE109091BE
:10222000930292FD10C098E0899F90011124262B03
:10223000209346020E94ED0B80914602859585957C
:1022400085950C940D110C94ED0B1092460280E0D4
:102250000C940D11209146028095822380934602B2
:10226000982F977099F430E0482F082E000C550BEA
:102270002417350759F09091930292FD07C0859578
:10228000859585950E940E0C0C9425110895CF9389
:102290009091930292FB222720F92817F9F0C82F7A
:1022A000892FC0FB82F980939302809192029091D2
:1022B00093020E94A31182E00E942A1180915F0282
:1022C00080FF0CC01F92CF9387E691E09F938F937E
:1022D0000E94C7050F900F900F900F90CF91089517
:1022E0008091930282FB882780F991E089270C94E2
:1022F000471181E00C94471180E00C94471180E075
:1023000090E00E94F62821E0893E9E4F09F020E0EF
:10231000822F089582E090E00C94EE2883E090E014
:102320000C94EE28CF9384E090E00E94EE28C82F12
:1023300082E290E00E94EE282C2F30E0A901582B79
:10234000CA01CF910895CF93C92F682F84E090E000
:102350000E94FC286C2F82E290E0CF910C94FC2824
:10236000AB01BC018FE090E00C940E29AB01BC01E5
:1023700083E190E00C940E2960E070E0CB010C94B6
:10238000B61160E070E0CB010E94B0110C94BC115A
:1023900069EE7EEF80E090E00E941A2960E082E022
:1023A00090E00E94FC2860E083E090E00E94FC281E
:1023B000109202021092030210920402109205027F
:1023C00060E084E090E00E94FC2860E082E290E01F
:1023D0000E94FC2860E085E090E00E94FC2860E01C
:1023E00086E090E00E94FC286FEF87E090E00E947A
:1023F000FC2840E050E0BA0188E090E00E940E29FD
:1024000060E08DE090E00E94FC2840E050E0BA01DE
:1024100088E190E00E940E2960E087E190E00E9450
:10242000FC2840E050E0BA018CE190E00E940E29C7
:1024300060E070E080E290E00E941A2940E050E005
:10244000BA0188E190E00E940E290C94C1110C940D
:10245000C811682F8EE090E00C94FC280E94CC20DC
:1024600060935B0270935C0280935D0290935E02C6
:1024700060935702709358028093590290935A02C6
:10248000089585B7806885BF85B7806885BF089542
:1024900081E008950C94481208950C944C120C9409
:1024A0004C120C944F120C944C120C9453120C942A
:1024B0004C120E94411281EF92E20E943F1F0E9443
:1024C00057120C9455120E944D120C944C120E94FB
:1024D00004150C94C8060E94B7200E9418160E948A
:1024E00067120C9451128F929F92AF92BF92CF922B
:1024F000DF92EF92FF920F931F93CF93DF93CDB7AD
:10250000DEB72A970FB6F894DEBF0FBECDBF0E948C
:102510002D16982E81110E942E1282E5A82E82E09F
:10252000B82E00E010E0802E802F0E942815D82EB3
:10253000F501C1905F01C826B1F40F5F1F4F053050
:10254000110589F78FEF89838A831B820E94C0203F
:102550008160782F9D838C8349815A816B818D8125
:102560000E940B072FC080915F0281FD0E942E15F3
:10257000E12CFF24F3948C2D8F21F1F00E944A125C
:10258000882399F0EE828F82DF2081E009F480E0D9
:1025900088870E94C0208160782F9A8789874E8122
:1025A0005F8168858A850E940B07F801EE5AFD4F0E
:1025B0008081F826F08206C0E394FF0CF3E0EF126E
:1025C000DACFBBCF81E0911001C080E02A960FB630
:1025D000F894DEBF0FBECDBFDF91CF911F910F9159
:1025E000FF90EF90DF90CF90BF90AF909F908F9033
:1025F00008950E9473120E94AE180C94D906CF93CE
:10260000DF930E942C14EC01811521E5920708F05C
:1026100045C0811530E5930708F094C0883E9105C8
:1026200028F5803E910508F0F8C0883A910570F4CD
:10263000853A910508F07CC08130910509F475C098
:1026400008F4E8C0049708F0E8C0E4C08F3B9105A7
:1026500008F0E0C0C85AD0E0CC0FDD1FC65BDE4FEB
:102660000990D881C02DCE019464D8C0811540E274
:10267000940758F4811551E0950708F0CEC08D3EBF
:10268000910508F4C7C09065C9C0C11580E4D8079A
:1026900008F4C0C0DF70CE01906AC0C0811525E586
:1026A0009207A8F4811534E5930708F095C08115C9
:1026B00043E5940708F07BC0811552E5950708F0C3
:1026C00061C0D82FCC27CE01816F906AA7C0C115F9
:1026D00089E5D807A0F4C11528E5D20708F082C023
:1026E000C11536E5D30708F095C08C2F0E94C014A1
:1026F0008F7190E0D82FCC27CE0190628FC0C1158A
:102700004AE5D40708F474C0CE0190568115904272
:1027100008F080C08D2F8F710E94C014DD27D06219
:102720008F71AE01582BCA0179C081E090E076C06C
:10273000C55AD0E0C858DE4F8881C82FD0E0CE01FE
:1027400090646CC074E0969587957A95E1F7282F90
:1027500023703C2F337081E090E002C0880F991FF6
:102760003A95E2F79C68AC01522B9A019C2F9F701E
:102770009695969550E2959FE0011124C9018C2B06
:102780009D2B4CC08370992721E030E002C0220FBE
:10279000331F8A95E2F79C2F9695969580E2989F35
:1027A000E0011124C22BD32BCE019C6837C083706B
:1027B000992721E030E002C0220F331F8A95E2F70B
:1027C0009C2F9695969540E2949FE0011124C22B90
:1027D000D32BCE019A6822C0D82FCC27CE01846F8C
:1027E000906A1CC0DC2FCC27CE01806F906A16C087
:1027F0008C2F8F700E94C01494E0D695C7959A953F
:10280000E1F7CF70D0E0DC2FCC27D0699E01282BD8
:10281000C90104C080E090E001C0CE01DF91CF91FA
:102820000895272F30E0F901EE0FFF1F2E0F3F1FF5
:10283000F9019FE0899FE00DF11D1124E60FF11DC4
:10284000EE0FFF1FE852FF4F8591949108950E946B
:1028500011140E94FF1208958238910569F1B0F4B5
:102860008133910509F46DC048F48932910509F46A
:1028700063C08A32910509F469C0089585339105D2
:1028800009F455C089339105B9F00895833E910547
:1028900069F138F4803E9105B1F0823E910509F16D
:1028A0000895863E9105A9F1873E9105B9F1843ED0
:1028B000910509F064C023C02091920220FD4FC011
:1028C00021FD4DC008958091920280FD44C0809109
:1028D000930280FF44C08091920284FD42C083EE47
:1028E0004DC08091920282FF38C0F5CF8091920254
:1028F00082FD33C08091930280FD31C0ECCF809186
:10290000930281FF32C08091920284FD2AC087EE3B
:1029100035C08091920283FF26C0F5CF809192024C
:1029200083FD21C08091930281FD1FC0ECCF809177
:10293000920285FD1CC01DC08091920285FD19C0C8
:1029400016C08091920286FD16C017C08091920237
:1029500086FD13C010C089E311C082EE0FC080EE67
:102960000DC080E00BC086EE09C084EE07C089E28E
:1029700005C085E303C08AE201C081E390E00895C9
:102980009091920292FF0DC0282F2871283019F4DF
:10299000877F846006C0282F2471243011F48B7F38
:1029A000886093FF0DC0282F2871283119F4877E85
:1029B000846106C0282F2471243111F48B7E886134
:1029C0002091930220FF0DC0382F3871383019F450
:1029D000877F816006C0382F3171313011F48E7FCE
:1029E000886021FF0DC0282F2871283119F4877EB7
:1029F000816106C0282F2171213111F48E7E8861FA
:102A000094FD877E089508950E947F11811102C070
:102A10000E9427120E948A1180935F020E949211E5
:102A200090939302809392020E9403150E948E114C
:102A3000682F70E080E090E00E948D0B6091FE01B5
:102A40007091FF0180910002909101020C94C50BDE
:102A5000E82FF0E0E756FD4F80810895CF92DF9296
:102A6000EF92FF920F931F93CF93DF938BE891E048
:102A70000E942E0589E9E82E82E0F82EC0E0D0E021
:102A800096E8C92E91E0D92E0EE711E0DF93CF939F
:102A9000DF92CF920E94C70583E891E00E942E0545
:102AA000F70181917F010E94AF061F928F931F93C0
:102AB0000F930E94C7058CE791E00E942E05219696
:102AC0008DB79EB708960FB6F8949EBF0FBE8DBF08
:102AD000C530D105D9F6DF91CF911F910F91FF90AD
:102AE000EF90DF90CF90089580EA8A95F1F70895EE
:102AF00000C008950C94741508950C947C150C94E2
:102B00007D150C947C150C948115F894E82FE295B2
:102B1000EF70F0E031A1282F2F7081E090E001C02C
:102B2000880F2A95EAF7982F9095932391A392A165
:102B3000892B82A378940895CF93DF93CEE7D1E0D9
:102B400089918F3F11F00E94851581E0C338D80725
:102B5000B9F784EF0E94851585EF0E94851586EFF1
:102B6000DF91CF910C948515CF92DF92EF92FF9277
:102B70000F931F93CF93DF938C01C62FD0E0CE012C
:102B800082589E4F7C01FC0190819F3F09F447C011
:102B9000D62EF894E92FE295EF70F0E081A19F70B6
:102BA00021E030E001C0220F9A95EAF7822B81A341
:102BB00082A12095282322A378940E947815EBE720
:102BC000F1E04EE751E031E0C12C21912F3F89F037
:102BD000A22FA295AF70B0E090968C9190E02F70EC
:102BE00002C0959587952A95E2F780FD02C0832F54
:102BF00001C080E0C82A330F4E175F0731F7F70195
:102C000080818F3F11F00E94851561E0C11001C0E5
:102C100060E08D2D0E947A15C00FD11FC882DF9110
:102C2000CF911F910F91FF90EF90DF90CF9008957B
:102C30000E949C1585E0E9E9F2E0DF01982F1D92E2
:102C40009A95E9F7E4E9F2E0DF011D928A95E9F748
:102C500085E00E9474160C942206FF920F931F9336
:102C6000CF93DF9300D000D01F92CDB7DEB78E0197
:102C70000F5F1F4F85E0F80111928A95E9F7F12C5B
:102C80006F2DC8010E94B415F394F5E0FF12F8CF40
:102C900045E050E0B80184E992E00E94E128FF2479
:102CA000F394009709F4F12C892B41F085E0F801A9
:102CB000A4E9B2E001900D928A95E1F72F2D45E04D
:102CC00069E972E084E992E00E9475160E94240688
:102CD0008F2D0F900F900F900F900F90DF91CF914D
:102CE0001F910F91FF9008950895FF920F931F93E6
:102CF000CF93DF938C01F62ED72FC42F222349F0D8
:102D000081E0809362020E94C020909361028093D0
:102D10006002809162028823C1F0809160029091EC
:102D200061020E94D820059780F0EF2DFD2FD80179
:102D30004C2F50E0CD01801B910B841795071CF49C
:102D40008D918193F7CF10926202DF91CF911F9105
:102D50000F91FF9008950E946D230E946B120C94B6
:102D600079230E947D230E94F9120C949B230E94D8
:102D70005E200E9454230E9459120E94AB160E94AA
:102D8000B1160E946312FBCF8091690280FF06C0DA
:102D90006091090170E0660F771F26C081FF04C0B3
:102DA0006091090184E005C082FF07C060910901BC
:102DB00088E0689FB001112417C0909168029923A0
:102DC000D1F060910801961788F72091090188E0F9
:102DD000289F90011124929FA001939F500D1124D0
:102DE00070E0CA010E94B3286038710540F4611593
:102DF000710519F406C068E070E0862F08958FE72A
:102E0000089581E008958091690280FF08C0609173
:102E1000050170E0759567957595679521C081FFEF
:102E200006C06091050170E07595679519C082FF35
:102E300004C06091050170E010C090916702992371
:102E400099F0609104019617A0F780910501899F80
:102E5000C001112470E00E94B3286038710540F46D
:102E60006115710519F406C061E070E0862F0895C0
:102E70008FE7089581E008958D3E21F40E94C416E5
:102E8000819504C08E3E29F40E94C41680936D0281
:102E900008958F3E21F40E94C416819504C0803F9E
:102EA00029F40E94C41680936C020895893F19F496
:102EB0000E94031705C08A3F31F40E9403178195D1
:102EC00080936E0208958B3F21F40E940317819531
:102ED00004C08C3F29F40E94031780936F02089569
:102EE0009FE0980F983078F421E030E0A90102C00B
:102EF000440F551F9A95E2F7CA0190916B02892BF6
:102F000080936B0208958D3F21F480916902816066
:102F10000BC08E3F21F480916902826005C08F3F13
:102F200029F48091690284608093690208958D3E3E
:102F300039F490916D0297FF35C010926D0259C01F
:102F40008E3E29F490916D021916BCF32BC090911E
:102F50006C028F3E29F497FF25C010926C0249C085
:102F6000803F19F41916CCF31DC090916E02893F71
:102F700029F41916BCF410926E023BC08A3F19F472
:102F800097FF10C0F8CF8B3F39F490916F0297FFF5
:102F900009C010926F022DC08C3F21F490916F02F6
:102FA0001916BCF39FE0980F983080F421E030E0D0
:102FB000A90102C0440F551F9A95E2F7CA018095F6
:102FC00090916B02892380936B0213C08D3F21F493
:102FD000809169028E7F0BC08E3F21F4809169023F
:102FE0008D7F05C08F3F29F4809169028B7F80938C
:102FF000690280916C02811106C080916D0281117D
:1030000002C01092680280916E02811106C0809108
:103010006F02811102C010926702089580915F02D1
:1030200083FF7EC081EC91E00E942E0580916B02AF
:103030001F928F938CEB91E09F938F930E94C70513
:103040008AEB91E00E942E0580916C02282F082EB9
:10305000000C330B3F938F9387EB91E09F938F93FB
:103060000E94C70585EB91E00E942E0580916D02BC
:10307000282F082E000C330B3F938F9382EB91E0A7
:103080009F938F930E94C70580EB91E00E942E05CD
:1030900080916E02282F082E000C330B3F938F93E4
:1030A0008DEA91E09F938F930E94C7058BEA91E090
:1030B0000E942E0580916F02282F082E000C330BE2
:1030C0003F938F9388EA91E09F938F930E94C70567
:1030D00085EA91E00E942E05809168021F928F93ED
:1030E00082EA91E09F938F930E94C70580EA91E066
:1030F0000E942E05809169021F928F938DE991E0C5
:103100009F938F930E94C7058AE991E00E942E0544
:103110008DB79EB74C960FB6F8949EBF0FBE8DBF6D
:103120000E94C02020916C02211104C020916D02E8
:10313000222321F0909366028093650220916E0213
:10314000211104C020916F02222321F09093640288
:10315000809363028AE692E00C949E1FEF92FF92A6
:103160000F931F93CF93DF9300D000D000D0CDB743
:10317000DEB786E0EAE6F2E0DE01119601900D92FC
:103180008A95E1F7E0906C02F0906D0200916E027A
:1031900010916F0210926C0210926D0210926E02EA
:1031A00010926F02E11003C0FF2009F45DC080910E
:1031B0006502909166020E94D820AC01909168024D
:1031C000992339F020910A0130E02417350758F08F
:1031D0004BC020910B018AE0289F900111242417F5
:1031E000350718F041C09F3F19F09F5F9093680228
:1031F000EE2061F00E94C4161E1414F09FEF01C06F
:1032000091E0989F902D112490936C02FF2061F023
:103210000E94C4161F1414F09FEF01C091E0989F04
:10322000902D112490936D0230916C023323E1F0C4
:1032300020916D022223C1F045EB3403C00111241B
:10324000992319F090936C0203C081E080936C0283
:1032500035EB2303C0011124992319F090936D02DB
:1032600003C081E080936D02011103C0112309F4B2
:103270005DC080916302909164020E94D820AC01ED
:1032800090916702992339F02091060130E02417CC
:10329000350758F04BC0209107018AE0289F900124
:1032A00011242417350718F041C09F3F19F09F5F84
:1032B00090936702002361F00E940317101614F028
:1032C0009FEF01C091E0989F902D112490936E0282
:1032D000112361F00E940317111614F09FEF01C033
:1032E00091E0989F902D112490936F0230916E027F
:1032F0003323E1F020916F022223C1F045EB340328
:10330000C0011124992319F090936E0203C081E04B
:1033100080936E0235EB2303C0011124992319F029
:1033200090936F0203C081E080936F0280916C02E2
:1033300081110BC080916D02811107C080916E02D6
:10334000811103C080916F0281110E940E18EB82DF
:10335000FC820D831E8386E0FE013196AAE6B2E070
:1033600001900D928A95E1F726960FB6F894DEBF8C
:103370000FBECDBFDF91CF911F910F91FF90EF90C6
:103380000895EAE6F2E086E0DF011D928A95E9F70A
:103390001092680210926702109269020895CF930A
:1033A000DF93EC01FB018281882309F43CC1C43026
:1033B000FDE5DF0760F4CB3F9CE5D90788F49E016B
:1033C00022503C452431310508F02EC109C0C236D7
:1033D000EDE5DE0729F0C63AFDE5DF0709F024C177
:1033E0000E9492119093930280939202C1318CE5D6
:1033F000D80709F4C6C008F042C0C930ECE5DE07C2
:1034000009F49BC000F5C5308CE5D80709F485C0E8
:1034100078F4C330ECE5DE0709F478C008F07AC030
:10342000C230DC4509F0F5C0809192028160EFC0A6
:10343000C7309CE5D90709F478C008F07AC08091BC
:1034400092028061E4C0CD30FCE5DF0709F487C05B
:1034500058F4CB309CE5D90709F479C008F07BC05B
:103460008091920288606FC0CF30FCE5DF0709F4DD
:1034700080C008F082C080919202877FC8C0CE3F92
:103480009CE5D90709F471C000F5C531FCE5DF07FB
:1034900009F485C068F4C3319CE5D90709F475C007
:1034A00008F095C00E94350B809192028F77AFC0D3
:1034B000CC3FFCE5DF07A9F108F054C0CB3FDC4569
:1034C00009F0A7C08091930240C0C230EDE5DE074D
:1034D00009F489C058F4C1158DE5D80709F45AC01C
:1034E00008F069C08091930282602FC0C236EDE57A
:1034F000DE0709F47CC0C63AFDE5DF0709F481C0A8
:10350000C330DD4509F085C080E06EC08091920235
:1035100082607DC08091920216C080919202886084
:1035200076C08091930282604FC080919202806247
:103530006EC08091920280646AC00E94350B8091B7
:103540009202806864C0846062C081603DC08091E6
:1035500092028E7F5CC0809192028D7F58C08091D4
:10356000920216C08091930218C0809193028D7FC1
:103570002BC0809192028F7E4AC0809192028F7DF3
:1035800046C0809192028F7B42C080919202877FD9
:103590008B7F3DC0809193028D7F8E7F15C080917F
:1035A000920282FB222720F991E0922790FB82F978
:1035B00090FB83F92CC080919302982F9095917085
:1035C0008E7F892B90FB81F98093930222C00E9409
:1035D000350B8091920287FB222720F991E09227F8
:1035E00090FB87F914C081E00E94291212C08091DB
:1035F000920284FB222720F991E0922790FB84F924
:1036000006C080919202982F909590FB80F980934C
:10361000920280919202909193020E94A3110E94C3
:10362000350B80E001C081E0DF91CF91089580915A
:1036300004011F928F93809105011F928F938091B7
:1036400008011F928F93809109011F928F9380919F
:103650000A011F928F9380910B011F928F9384EE2A
:1036600091E09F938F930E94C7058DB79EB70E96EA
:103670000FB6F8949EBF0FBE8DBF0895883220F517
:103680008E3108F068C08B3091F1C0F4873009F0BA
:10369000BEC081E080930B0184E180930A018AE03F
:1036A000809309018EE18093080188E080930501F1
:1036B00088E28093040186E493E0C6C0833109F474
:1036C00043C0843169F1A3C08F3409F49EC028F44B
:1036D000893231F1883359F09AC0813531F008F4DC
:1036E000D4C0823509F4A7C092C08FEFA5C088E688
:1036F00093E00E942E050E94171B1F9281E08F937A
:103700001F9288E08F9381E692E09F938F930E94AF
:10371000C7050F900F900F900F900F900F9096C0CD
:1037200085E693E00E942E0580917402882309F4B7
:10373000AAC0109274021092730210927202109238
:10374000710210927002B1C087E593E00E942E05CD
:103750000E94171B7BC08D5180937402833031F11E
:1037600070F48130D1F0823009F03FC08AE091E0FE
:10377000909373028093720280E991E01FC08530BC
:1037800059F108F1863089F584E091E09093730255
:10379000809372028BEC91E011C08BE091E09093EA
:1037A00073028093720287E891E008C089E091E09B
:1037B00090937302809372028CE991E0909371026E
:1037C0008093700218C088E091E090937302809318
:1037D000720289EA91E0F2CF85E091E09093730262
:1037E0008093720288EB91E0E9CF1092740284E535
:1037F00093E00E942E0580917402882309F455C03D
:103800001F928F9380E593E00DC08AE015C083E49A
:1038100093E01AC097FF47C0108280811F928F9358
:103820008DE393E09F938F930E94C7050F900F90B5
:103830000F900F900BC081E0E0917202F091730243
:10384000309729F58AE393E00E942E0520917402B7
:10385000222359F18091700290917102009711F426
:1038600083E891E09F938F931F922F9381E393E0DE
:103870009F938F930E94C7050F900F900F900F900A
:103880000F900F9016C080E0089586EFD5CF20816D
:10389000082E000C990B820F911D8F3F910509F0A6
:1038A0000CF4B8CF8FEF8083B8CF8DE293E00E9405
:1038B0002E0581E00895CF93C82F1F928F938EE736
:1038C00093E09F938F930E94C70581E090E0A0E072
:1038D000B0E0BC01CD0104C0660F771F881F991F9F
:1038E000CA95D2F70E948D0B0F900F900F900F90FA
:1038F000CF910C94350BEF92FF920F931F93CF93C0
:10390000DF938B3109F4EDC008F08EC08B3009F4E1
:10391000B1C008F078C0863009F4AFC020F485301B
:1039200009F4BDC04EC1873009F4C0C0883009F029
:1039300048C10E948E111F928F9382EA97E09F9355
:103940008F930E94C7050E948A1183FB992790F9E3
:103950001F929F9382FB992790F91F929F9381FB5F
:10396000992790F91F929F93982F91701F929F9380
:103970001F928F9389E597E09F938F930E94C705CD
:103980000E94921187FB222720F91F922F9386FB1A
:10399000222720F91F922F9385FB222720F91F92BF
:1039A0002F9384FB222720F91F922F9383FB22273A
:1039B00020F91F922F9382FB222720F91F922F9329
:1039C00091FB222720F91F922F93292F21701F92FC
:1039D0002F9381FB222720F91F922F93282F2170EC
:1039E0001F922F939F938F9384E796E09F938F93DB
:1039F0000E94C7058DB79EB788960FB6F8949EBFF4
:103A00000FBE8DBF35C0803109F495C020F48E30D3
:103A100009F47BC0D6C0863109F4A8C0893109F009
:103A2000D0C08EEE93E084C08A32E1F060F4873239
:103A300009F4C3C028F48E3108F4C3C08D51BEC050
:103A4000893269F1BEC0833448F48A3308F0B3C0C8
:103A5000853309F4B2C0883369F0B3C0833409F404
:103A6000ACC0AFC08DE498E00E942E050E942712E2
:103A7000C1E0ACC081ED94E05BC080915F02817FCA
:103A80008E7F80935F028AEA94E00E942E0589E48B
:103A900098E00E942E0581E080937502E9CF8DE2C7
:103AA00098E00E942E050E942706E2CF80915F02D7
:103AB000C82FC095C170C0FB80F980935F02CC23F2
:103AC00029F081E298E00E942E0580C084E198E010
:103AD0000E942E0580915F02897F877F80935F021D
:103AE000C7CF90915F0291FBCC27C0F981E0C82736
:103AF000892FC0FB81F980935F02CC2319F087E006
:103B000098E029C089EF97E013C090915F0292FB83
:103B1000CC27C0F981E0C827892FC0FB82F98093A8
:103B20005F02CC2319F08AEE97E015C08AED97E08A
:103B30000E942E059DCF90915F0293FBCC27C0F988
:103B400081E0C827892FC0FB83F980935F02CC23D3
:103B500051F08EEC97E00E942E0580915F0281600B
:103B600080935F0233C081EC97E0E2CF0E94CC20CB
:103B7000162F072FF82EE92ED0919102C09118012F
:103B80000E94491FEF92FF920F931F931F92DF93A2
:103B90001F92CF931F928F9383E893E09F938F930D
:103BA0000E94C7058DB79EB70C960FB6F8949EBFBE
:103BB0000FBE8DBF5DCF895301C080E00E945B1CAA
:103BC00057CF8FEB97E00E942E05C0E08C2FDF913E
:103BD000CF911F910F91FF90EF90089580E008958D
:103BE0000C94EE1DCF93C82F80917502813071F037
:103BF00040F0823009F045C08C2F0E943E1B81E0CE
:103C000046C00E9488108232F1F504C00E948810DC
:103C1000823261F48C2F0E94F01D811104C08C2F20
:103C20000E947B1C2CC081E090E029C08C2F0E9458
:103C3000EE1D811123C0C431C9F058F4CB3069F0B6
:103C4000C031B9F482E08093750288E30E943E1B84
:103C500015C0C93259F0C83361F48AEA94E00E9471
:103C60002E058AE793E00E942E0508C01092750287
:103C70000CC088E793E00E942E0507C081E08170A8
:103C800006C01092750280E002C080E0F8CFCF91AC
:103C90000895CF93DF9386319C4541F5EB010E9457
:103CA0008810982F8A812091020130910301882386
:103CB00079F09A7A81E009F480E08093760291119C
:103CC00002C069E201C065E3C9010E941A200AC06E
:103CD00080917602811102C069E201C065E3C901E9
:103CE0000E941C200E94CA1080E001C081E0DF9188
:103CF000CF9108950F931F93CF93DF93C42FD22FAB
:103D0000FC0182818823C9F0409379020E94C0207F
:103D1000909378028093770280E28C0F883008F0CD
:103D200057C0C77081E001C0880FCA95EAF7DF91DC
:103D3000CF911F910F910C949208809179024813B2
:103D400030C080917702909178020E94D820883C00
:103D5000910538F510E21D0FCD17B9F080E28C0FF8
:103D6000883040F4C77081E001C0880FCA95EAF737
:103D70000E949908183028F581E09D2F977001C0A6
:103D8000880F9A95EAF70E949208802F0E9489086E
:103D90001830F0F4D77081E001C0880FDA95EAF7A7
:103DA0000AC080E28C0F883098F4C77081E001C0AF
:103DB000880FCA95EAF7DF91CF911F910F910C946C
:103DC0009908802FDF91CF911F910F910C94890852
:103DD000DF91CF911F910F9108950F939C01CB011B
:103DE000243F4CE5340731F188F4293DFCE53F07D9
:103DF000D9F02A3D4CE5340779F1283D3C45A9F539
:103E000006E221EE41EE68ED7CE52BC0263FFCE5A5
:103E10003F07E1F0A8F0273F3C4539F507E225EEE2
:103E200046EE67EF7CE51DC007E225EE45EE69ED45
:103E30007CE517C006E221EE40EE64EF7CE511C0A0
:103E400007E225EE44EE65EF7CE50BC006E221EECD
:103E500042EE66EF7CE505C008E221E045EE6AED42
:103E60007CE50E947A1E80E008C0FC0182818823E4
:103E700019F01092790201C081E00F91089590939A
:103E8000F1018093F001089590937F0280937E0268
:103E90000895E0917E02F0917F02309721F0019029
:103EA000F081E02D099480E00895EF92FF920F9346
:103EB0001F93CF93DF93E0917E02F0917F023097C2
:103EC000B1F18C010280F381E02D099580915F02B0
:103ED00082FF2DC080FF04C086E698E00E942E0578
:103EE000E80118E080E6E82E88E0F82E80915F0275
:103EF00080FF0BC088811F928F93FF92EF920E94E8
:103F0000C7050F900F900F900F901150219611112F
:103F1000EDCF80915F0280FF0AC08EE598E0DF91CF
:103F2000CF911F910F91FF90EF900C942E05DF9190
:103F3000CF911F910F91FF90EF900895E0917E0235
:103F4000F0917F02309739F022E0DC012C9304805D
:103F5000F581E02D0994089520917C0230917D0235
:103F60002817390771F090937D0280937C02E091CD
:103F70007E02F0917F02309721F00680F781E02DDC
:103F80000994089520917A0230917B02281739070D
:103F900071F090937B0280937A02E0917E02F0911F
:103FA0007F02309721F00084F185E02D0994089577
:103FB000FC01329697E080E0915029F02191222374
:103FC000D9F38F5FF9CF0895662349F0FC0132964B
:103FD00008962191621729F0E817F907D1F780E0D8
:103FE000089581E008959C01FC0132969FEF80E0E6
:103FF0004191461789F09F3F19F4411101C0982F54
:104000008F5F8630A9F79F3F39F0F901E90FF11D65
:1040100097FDFA956283089508959C012A5F3F4FAA
:10402000FC014281461301C0128201968217930758
:10403000B9F708950C94F31F0C940D20029626E016
:10404000FC0111922A95E9F7089508950C94252012
:1040500083E0809380020C942620811102C081E0CD
:1040600001C082E0809380020C9426200C942D20C5
:1040700081E0809380020C9426200C9438200895CF
:104080000C943F200C9440200C943F200C943F2033
:104090000C943F20CF930E9446200E942D160E9430
:1040A0004420C0E08C2F0E942815811104C0CF5FEE
:1040B000C530C1F701C081E0CF91089508951F92E6
:1040C0000F920FB60F9211248F939F93AF93BF93CC
:1040D00080918102811113C080919E0290919F0274
:1040E000A091A002B091A1024196A11DB11D8093A3
:1040F0009E0290939F02A093A002B093A102BF9151
:10410000AF919F918F910F900FBE0F901F901895B8
:104110008091A602843031F10E94A706109281029C
:1041200020E488E190E00FB6F894A89580936000B1
:104130000FBE2093600083B7817F846083BF83B705
:10414000816083BF7894889583B78E7F83BF0FB6D5
:10415000F894A89580916000886180936000109227
:1041600060000FBE08950E94350B0C94AB0682E0F0
:1041700084BD93E095BD9AEF97BD80936E0008953E
:104180002FB7F89480919E0290919F02A091A00277
:10419000B091A1022FBF08952FB7F89460919E02AD
:1041A00070919F028091A0029091A1022FBF08956B
:1041B0009C014FB7F89480919E0290919F02A0912C
:1041C000A002B091A1024FBF821B930B0895789477
:1041D0001F920F920FB60F9211248F939F93AF935C
:1041E000BF9380919E0290919F02A091A002B091F6
:1041F000A1020196A11DB11D80939E0290939F0282
:10420000A093A002B093A102BF91AF919F918F9113
:104210000F900FBE0F901F90189587E797E7909328
:104220000108809300089AE088E10FB6F894A895F9
:10423000809360000FBE90936000FFCF809190024A
:104240000895089522E02093E9002FEF3091E800CF
:10425000215035FD06C035ED3A95F1F700002111EA
:10426000F5CF2091E80025FF0BC040E050E066E06C
:1042700070E00E940A248091E8008E778093E80025
:104280000895CF93DF9321E02093E9002FEF309141
:10429000E800215035FD06C035ED3A95F1F70000F4
:1042A0002111F5CF2091E80025FF14C0EC0140E07A
:1042B00050E068E070E00E940A248091E8008E7768
:1042C0008093E80088E0FE01A8E8B2E001900D923A
:1042D0008A95E1F7DF91CF910895809384027093DE
:1042E0008602609385028091A602843001F582E007
:1042F0008093E9008FEF9091E800815095FD06C012
:1043000095ED9A95F1F700008111F5CF8091E800C5
:1043100085FF0DC040E050E063E070E084E892E08B
:104320000E940A248091E8008E778093E800089527
:10433000BC0184E00C946D21BC0183E00C946D21E0
:104340008CE898E00E942E058091A502811109C099
:104350000E949B250E94F8258091E2008460809352
:10436000E200089588E898E00E942E051092A502C8
:10437000089584E898E00E942E050C943D2080E882
:1043800098E00E942E056091A20281E0611101C0B7
:1043900080E00C9428208CE798E00E942E059091F4
:1043A000A60281E0943009F080E06091A2020C94B2
:1043B0002D20209183022F5F822F62E30E94A72885
:1043C000992319F02093830208951092830280911B
:1043D0008702882371F18091A602843041F5809193
:1043E000E9008F702091EC00922F917020FD90E8F1
:1043F000892B93E09093E9009091EB0090FF14C01B
:104400009091EE0097FF10C09091E80095FF03C0D7
:104410001092F100F9CF9091E80090FF05C09091C3
:10442000E8009E779093E8008F708093E9001092E7
:104430008702089542E061EC81E00E94142542E287
:1044400061EC82E00E94142542E261EC83E00E946C
:1044500014259091A60281E0943009F080E06091EB
:10446000A2020C9436208091A802833009F461C026
:1044700030F4813071F0823009F49AC008958A30A6
:1044800009F486C08B3009F46CC0893009F0A8C0EB
:1044900020C08091A702813A09F0A2C08091E80073
:1044A000877F8093E8008091AB029091AC02892BCA
:1044B00021F468E088E892E003C060E080E090E0EA
:1044C00070E00E9455248091E8008B778093E8008B
:1044D00008958091A702813209F082C08091AB02D9
:1044E0009091AC02029708F07BC08091E800877F32
:1044F0008093E8008091E80082FD05C08091A602CB
:104500008111F8CF6DC02091F3008091F20090E00E
:10451000922B029731F48091F100813011F08630B6
:1045200021F48091F100809390028091E8008B77D4
:1045300053C08091A702813A09F052C08091AB022A
:104540009091AC02892B09F04BC08091E800877FE5
:104550008093E8008091E80080FFFCCF80911801F3
:1045600036C08091A7028132D9F58091AB0290913B
:10457000AC02892BA9F58091E800877F8093E80041
:104580000E9449258091A902809318010C94350B53
:104590008091A702813221F58091E800877F809386
:1045A000E8000E9449258091AA0280939102089513
:1045B0008091A702813AA1F48091E800877F8093DF
:1045C000E8008091E80080FFFCCF80919102809309
:1045D000F1008091E8008E778093E8000C944925E3
:1045E00008959FB7F894109287029FBF9091A602FA
:1045F000943009F057C09091E9009F703091EC0021
:10460000232F217030FD20E8922B23E02093E90036
:104610002091EB0020FF43C02091EE0027FF3FC018
:1046200020918202222321F02091E80025FF37C04B
:104630001092820226E03091E80035FD15C03091DD
:10464000A602343061F53091EB0035FD28C02150D1
:1046500021F481E08093820222C0EFE9FFE03197EC
:10466000F1F700C00000E7CF8093F1008091E800EF
:1046700085FD0AC08091E80080FFFCCF8091E800B2
:104680008E778093E80006C08FB7F89421E02093DE
:1046900087028FBF9F709093E90080E008959F701C
:1046A0009093E9008FEF089584B7877F84BF0FB69A
:1046B000F894A895809160008861809360001092C2
:1046C00060000FBE90E080E80FB6F8948093610020
:1046D000909361000FBE0C9438200E949B250E948D
:1046E000F825E2EEF0E080818460808378940C9479
:1046F0008C288CE091E00C94441F8091A6028530B8
:10470000C9F488E798E00E942E058091A6028530C2
:1047100079F40E9488208091A4028823B1F30E943A
:104720004A20882391F30E94F4230E94350BEDCF99
:104730000C94B320089508950C949E23292F3327B9
:1047400023303105C9F060F42130310581F0223089
:10475000310509F041C08BE590E02CEB38E040C01A
:1047600021323105E1F02232310531F135C082E1EB
:1047700090E027E139E034C099278130910549F074
:1047800028F0029749F5E0E9F8E005C0E8EBF8E029
:1047900002C0EEE9F8E0849190E09F0121C063300F
:1047A0007105D0F4660F771FFB01E751FE4F2081A2
:1047B000318189E090E014C06330710568F4FB0139
:1047C000EE0FFF1FED51FE4F20813181FB01E052C2
:1047D000FE4F808190E004C080E090E020E030E077
:1047E000FA0131832083089580E189BD82E189BD8A
:1047F00009B400FEFDCF8091D8008F7D8093D80052
:104800008091E00082608093E0008091E00081FD73
:10481000FCCF0895CF92DF92EF92FF920F931F93F8
:10482000CF93DF93EC018B017A010E9468258111FF
:1048300033C0E114F10439F0F70180819181081B44
:10484000190BC80FD91FC12CD12C0115110519F155
:104850008091E80085FD16C08091E8008E778093F6
:10486000E800E114F10449F0F70180819181C80E5C
:10487000D91ED182C08285E00FC00E94682588239E
:1048800021F30AC089918093F10001501109FFEFD3
:10489000CF1ADF0ADACF80E0DF91CF911F910F911D
:1048A000FF90EF90DF90CF9008952091AD0230916E
:1048B000AE022617370748F06115710539F42091CB
:1048C000E8002E772093E80001C0B901FC0120E048
:1048D0006115710579F18091A6028823F1F1853087
:1048E000F1F18091E80083FD3CC08091E80082FDF9
:1048F0002EC08091E80080FFEBCF2091F3008091E3
:10490000F20090E0922B6115710551F0883091050D
:1049100038F421912093F100615071090196F3CF91
:1049200021E0089709F020E08091E8008E778093DD
:10493000E800CECF2111CFCF0AC08091A6028823F4
:1049400061F0853061F08091E80083FD0AC08091BC
:10495000E80082FFF2CF80E0089582E0089583E0CE
:10496000089581E008952091AD023091AE0226179E
:10497000370748F06115710539F42091E8002E776A
:104980002093E80001C0B901FC0120E06115710528
:1049900091F18091A602882309F440C0853009F482
:1049A0003FC08091E80083FD3DC08091E80082FD1A
:1049B0002FC08091E80080FFE9CF2091F300809123
:1049C000F20090E0922B6115710559F08830910545
:1049D00040F424912093F1003196615071090196C1
:1049E000F2CF21E0089709F020E08091E8008E776F
:1049F0008093E800CBCF2111CCCF0AC08091A602D2
:104A0000882361F0853061F08091E80083FD0AC061
:104A10008091E80082FFF2CF80E0089582E008955F
:104A200083E0089581E00895982F973068F590937A
:104A3000E900981739F07091EC002091ED00509149
:104A4000F00003C0242F762F50E021FD02C09F5FAD
:104A5000ECCF3091EB003E7F3093EB003091ED00D6
:104A60003D7F3093ED003091EB0031603093EB00EF
:104A70007093EC002093ED005093F0002091EE0035
:104A800027FDE5CF80E008958F708093E90081E0F5
:104A900008958091A70287FF11C08091E80082FDF0
:104AA00005C08091A6028111F8CF11C08091E80065
:104AB0008B770BC08091A602882349F08091E80093
:104AC00080FFF8CF8091E8008E778093E80008950A
:104AD0002091E4003091E50095E64091EC00842FB0
:104AE000817040FF23C08091E80080FD1DC080914F
:104AF000A602882399F0853099F08091EB0085FD1E
:104B000011C04091E4005091E5002417350729F3C6
:104B1000915011F09A01E1CF84E0089582E0089568
:104B200083E0089581E0089580E008954091E800D1
:104B300042FFDDCF08950E9409260E941126E0EE73
:104B4000F0E0808181608083E8EDF0E080818F7704
:104B5000808319BCA7EDB0E08C918E7F8C9380810F
:104B60008F7E80831092A50208950F931F93CF9399
:104B7000DF930E9409260E941126C8EDD0E08881AB
:104B80008F77888388818068888388818F7D8883F8
:104B900019BC1092A6021092A2021092A4021092C6
:104BA000A30200EE10E0F80180818B7F8083888172
:104BB0008160888342E060E080E00E941425E1EE9D
:104BC000F0E080818E7F8083E2EEF0E08081816082
:104BD0008083808188608083F80180818E7F8083DC
:104BE000888180618883DF91CF911F910F91089513
:104BF000E8EDF0E080818F7E8083E7EDF0E080815A
:104C00008160808384E082BF81E08093A5020C9460
:104C1000B525E8EDF0E080818E7F80831092E20080
:104C200008951092DA001092E10008951F920F92F9
:104C30000FB60F9211242F933F934F935F936F936F
:104C40007F938F939F93AF93BF93EF93FF93809145
:104C5000E10082FF0BC08091E20082FF07C08091DB
:104C6000E1008B7F8093E1000E94D9218091DA00DE
:104C700080FF1FC08091D80080FF1BC08091DA00A8
:104C80008E7F8093DA008091D90080FF0DC080E193
:104C900089BD82E189BD09B400FEFDCF81E080932A
:104CA000A6020E94A02105C019BC1092A6020E9473
:104CB000B2218091E10080FF19C08091E20080FF65
:104CC00015C08091E2008E7F8093E2008091E20027
:104CD00080618093E2008091D80080628093D80048
:104CE00019BC85E08093A6020E94BF218091E1005B
:104CF00084FF30C08091E20084FF2CC080E189BD38
:104D000082E189BD09B400FEFDCF8091D8008F7D7E
:104D10008093D8008091E1008F7E8093E1008091A4
:104D2000E2008F7E8093E2008091E20081608093B8
:104D3000E2008091A202882311F084E007C08091F4
:104D4000E30087FD02C081E001C083E08093A602FA
:104D50000E94CB218091E10083FF29C08091E20075
:104D600083FF25C08091E100877F8093E10082E08E
:104D70008093A6021092A2028091E1008E7F809320
:104D8000E1008091E2008E7F8093E2008091E2005A
:104D900080618093E20042E060E080E00E941425A0
:104DA0008091F00088608093F0000E94B921FF910B
:104DB000EF91BF91AF919F918F917F916F915F9193
:104DC0004F913F912F910F900FBE0F901F9018950C
:104DD0001F920F920FB60F9211242F933F934F9370
:104DE0005F936F937F938F939F93AF93BF93CF9373
:104DF000DF93EF93FF93C091E900CF708091EC00B7
:104E0000D82FD17080FDD0E81092E9008091F00099
:104E1000877F8093F00078940E942C271092E900FD
:104E20008091F00088608093F000CD2BCF70C0930C
:104E3000E900FF91EF91DF91CF91BF91AF919F91E9
:104E40008F917F916F915F914F913F912F910F9033
:104E50000FBE0F901F9018951F93CF93DF93CDB780
:104E6000DEB7AA970FB6F894DEBF0FBECDBFE7EA54
:104E7000F2E08091F100819322E0EF3AF207C9F766
:104E80000E9433228091E80083FF2EC18091A70207
:104E90009091A802492F50E04A30510508F024C1F2
:104EA000FA01EE59FF4F0C94C728803821F0823860
:104EB00009F01AC108C08091A3029091A40299231D
:104EC00089F082600FC08091AB028F70873008F04C
:104ED0000BC18093E9008091EB0085FB882780F966
:104EE0001092E9009091E800977F9093E8008093FA
:104EF000F1001092F100D1C0282F2D7F09F0F4C0ED
:104F0000882319F0823061F0EFC08091A9028130CE
:104F100009F0EAC0933009F080E08093A4022EC02B
:104F20008091A90281112AC08091AB028F702FEF6E
:104F3000280F263008F0D8C08093E9002091EB00BC
:104F400020FF1CC0933021F48091EB00806214C0DC
:104F50009091EB0090619093EB0021E030E0A9018B
:104F600002C0440F551F8A95E2F74093EA00109261
:104F7000EA008091EB0088608093EB001092E900DA
:104F80008091E800877F8093E8000E944925ACC0AB
:104F90008111AAC01091A9021F778091E300807847
:104FA000812B8093E3008091E800877F8093E80065
:104FB0000E9449258091E80080FFFCCF8091E300AA
:104FC00080688093E300111102C082E001C083E099
:104FD0008093A60289C08058823008F085C08091F5
:104FE000A9029091AA028C3D53E0950779F583E0E0
:104FF0008A838AE289834FB7F894DE01139620E012
:105000003EE051E2E32FF0E050935700E49120FF9F
:1050100003C0E295EF703F5FEF708E2F90E0EA30B3
:1050200010F0C79601C0C0968D939D932F5F2431D9
:1050300049F74FBF8091E800877F8093E8006AE2DC
:1050400070E0CE0101960E94552416C06091AB021B
:105050007091AC02AE014F5F5F4F0E949C23BC0178
:10506000892B09F441C09091E800977F9093E80064
:1050700089819A810E94B3248091E8008B77809384
:10508000E80032C0803881F58091E800877F809306
:10509000E8008091A2028093F1008091E8008E7771
:1050A00072CF811121C08091A9029091AA02992703
:1050B0000297D4F48091E800877F8093E800809184
:1050C000A9028093A2020E9449258091A202811127
:1050D00006C08091E30087FD02C081E001C084E04A
:1050E0008093A6020E941A228091E80083FF0AC0E2
:1050F0008091E800877F8093E8008091EB008062D8
:105100008093EB00AA960FB6F894DEBF0FBECDBF1A
:10511000DF91CF911F910895CF938091A6028823AC
:10512000A1F0C091E900CF709091EC00892F8170BF
:1051300090FD80E8C82B1092E9008091E80083FD83
:105140000E942C27CF70C093E900CF910895991B3E
:1051500079E004C0991F961708F0961B881F7A956E
:10516000C9F78095089597FB072E16F4009407D091
:1051700077FD09D00E94CD2807FC05D03EF490951C
:1051800081959F4F0895709561957F4F0895EE0F1B
:10519000FF1F0590F491E02D0994AA1BBB1B51E160
:1051A00007C0AA1FBB1FA617B70710F0A61BB70B97
:1051B000881F991F5A95A9F780959095BC01CD013C
:1051C0000895FB01DC0104C08D910190801921F448
:1051D00041505040C8F7881B990B0895F999FECFAC
:1051E00092BD81BDF89A992780B50895A8E1B0E0F5
:1051F00042E050E00C942229262FF999FECF92BD6F
:1052000081BDF89A019700B4021639F01FBA20BD8B
:105210000FB6F894FA9AF99A0FBE08950396272FBD
:105220000E94FD280E94FC28252F0E94FD28242F83
:105230000C94FD280196272F0E94FD280C94FC2831
:10524000DC01CB01FC01F999FECF06C0F2BDE1BD46
:10525000F89A319600B40D9241505040B8F7089535
:04526000F894FFCFF0
:10526400C8004802280850011E0A14011E214121C9
:1052740022219C219821212101E200E900EA00B5C4
:1052840000B600B700CD008301CC008A01920194DE
:10529400012102230224022502260227022A02B344
:1052A40000B4006F007000818283E200E900EA002C
:1052B400B500B600B700CD008301CC008A0192018D
:1052C40094012102230224022502260227022A0233
:1052D400B300B4006F007000818283F4F5F6946625
:1052E40097C6343F3F3F006D6B5F64656C61790026
:1052F4006D6B5F696E74657276616C006D6B5F6D6A
:1053040061785F7370656564006D6B5F74696D656A
:105314005F746F5F6D6178006D6B5F776865656C56
:105324005F6D61785F7370656564006D6B5F77684E
:1053340065656C5F74696D655F746F5F6D6178003E
:10534400407B22C6094B092909CE08E70800090059
:00000001FF
